:020000040000FA
:040000006CEF00F0B1
:0800080071D00B6E040E056EB1
:100010000C500A5C02E10B50095C040ED8B0010ED2
:10002000D8B4020E0514D8A4010E12000F0EEA6E09
:1000300002C0E9FF031CE988E92AEC1609500A10FE
:10004000D8B412003AD802C0E9FF0350EF1A0000FA
:1000500000D000D0092AD8B40A3EF9D7EF1A12000E
:10006000E836E8363C0B0109C212C009C216C0507E
:10007000F80B0309C06E320E15D8C282C2B2FED789
:10008000C4CF11F0C350106E12000C6A0B6EFF0E3D
:100090000B260C2200D0D8A01200030E0A6EE70E29
:1000A00002D8F5D70A6AFE0F096EE86A0A5AD8A084
:1000B00012000000090600D0F8D7091E0A1E094ADE
:1000C0000A2A12000A6A0C6AA0DF04E00CC00AF0D7
:1000D0000BC009F009501200F86A006A4F0EAF6EAB
:1000E000240EAC6E900EAB6E000159D09EAA1BD0B0
:1000F000060EAB1412E1E1CF57F0E2CF58F0592AC7
:1001000015EE00F05950E126000EE222AECFE7FFD7
:1001100057C0E1FF58C0E2FF1100AE50AE50AB989F
:10012000AB8811000AD0F2A408D0F294164A172A1C
:10013000817A156AD6CF14F01100110059505A5C1B
:1001400014E05A2AE9CF09F0EACF0AF005EE00F0F0
:100150005A50E926000EEA22EF50096E09C0E9FF65
:100160000AC0EAFFD880120004D0E868096ED8A05F
:1001700012001200596A5A6A9D8AF28EF28C12009D
:100180009D9A05EE00F0000EEE6AE82EFDD7596A42
:100190005A6A9D8A12009EA8FED7AD6E1200730E99
:1001A000926EE00E936EC00E946EC16E94968B9616
:1001B00094908B90949A8B8A94988B8893908A9041
:1001C00093928A92939A8A9A9288928A9296899620
:1001D00092948994526A266A276A939A8A8A640E4C
:1001E00054DF939A8A9AC6DFCBDFD56AF294F28AFB
:1001F000870ED56EC26A0D0EC16E820EC06EC280B1
:10020000D6EC04F0030E0C6EE80E40DFFFEC05F0B8
:10021000C80E3BDF93DF186ECD0E185C07E3FE0EB1
:10022000185C02E31CD102D0196A19D118AE19D09A
:10023000196A8C0E185C05E118C019F01A681B6861
:100240000FD09C0E185C05E118C019F01C681D68E1
:1002500007D0BC0E185C04E118C019F01E681F68B6
:10026000FED0195202E1FBD0FAD08C0E195C1EE1CF
:100270001A2803E118C01AF017D018C01BF0790E25
:100280001A5C04E152928B9626960DD07A0E1A5C77
:1002900004E1529426988B9006D07B0E1A5C03E101
:1002A000529026948A921A68DAD0D9D09C0E195CA2
:1002B000D8A4C9D01C2803E118C01CF0C2D018C0B3
:1002C0001DF01D5216E1790E1C5C04E15292269637
:1002D0008B960DD07A0E1C5C04E1529426988B907C
:1002E00006D07B0E1C5C03E1529026948A921C6817
:1002F000B6D0790E1C5C34E152828B867F0E1D5C79
:100300002DE226861D1C086E7F0E0814106E116AE1
:1003100010C007F0066AD890073606C061F007C023
:1003200062F0D6CF14F0D7CF15F061C006F062C0EE
:1003300007F006501424226E07501520236E000E7D
:100340001620246E000E1720256E24C06BF025C0E9
:100350006CF022C075F023C076F001D0269670D0E4
:100360007A0E1C5C34E152848B807F0E1D5C2DE282
:1003700026881D1C086E7F0E0814106E116A10C0AE
:1003800007F0066AD890073606C063F007C064F02D
:10039000D6CF14F0D7CF15F063C006F064C007F0D5
:1003A00006501424226E07501520236E000E1620CE
:1003B000246E000E1720256E24C06DF025C06EF04F
:1003C00022C077F023C078F001D0269839D07B0E78
:1003D0001C5C34E152808A827F0E1D5C2DE22684F3
:1003E0001D1C086E7F0E0814106E116A10C007F0F5
:1003F000066AD890073606C05FF007C060F0D6CF17
:1004000014F0D7CF15F05FC006F060C007F00650BB
:100410001424226E07501520236E000E1620246E21
:10042000000E1720256E24C069F025C06AF022C096
:1004300073F023C074F001D0269402D01C680FD052
:100440001C680DD00CD0BC0E195C09E11E2803E11C
:1004500018C01EF003D018C01FF0AAD900D03A521D
:10046000D8B44ED0D6CF4EF0D7CF4FF04B504F1818
:10047000010B1EE04B804FA04B903A04096E02081E
:1004800017E3FA6AD8900936FA360936FA36A40E16
:100490000926040EFA220500040EFE6EB00EFD6E53
:1004A0000950F96E2DEF08F0AEEF08F025EF09F0D6
:1004B000D6CF4EF0D7CF4FF0E86A4BB2010F4FBE08
:1004C00001081EE04B824FAE4B923A04096E0208BF
:1004D00017E3FA6AD8900936FA360936FA36F40E76
:1004E0000926040EFA220500050EFE6E000EFD6EB2
:1004F0000950F96E9CEF09F0EBEF09F044EF0AF0B8
:10050000040E3B5CD8A0BED03BA429D0D6CF4EF081
:10051000D7CF4FF04B504F18040B21E04B844FA422
:100520004B9430502E5C106E31502F58116E7F0E50
:100530001014206E30502E5C106E31502F58116EFA
:1005400010C021F011C0F3FF070EF3322132E82E64
:10055000FCD7E20E20DE20501EDE21501CDE3BA622
:1005600025D0D6CF4EF0D7CF4FF0E86A4BB6010F6B
:100570004FB001081BE04B864FA04B96000E30ECAD
:1005800000F0426E11C043F042C021F043C0F3FFBF
:10059000070EF3322132E82EFCD77F0E4214206E74
:1005A000E30EF9DD2050F7DD2150F5DD3BA828D022
:1005B000D6CF4EF0D7CF4FF0E86A4BB8010F4FB00F
:1005C00001081EE04B884FA04B98010E30EC00F064
:1005D000426E11C043F042C021F043C0F3FF070E4A
:1005E000F3322132E82EFCD77F0E4214206EE40E47
:1005F000CBEC00F02050CBEC00F02150CBEC00F025
:100600003BAA10D0D6CF4EF0D7CF4FF07F0E4E146E
:10061000206EE50ECBEC00F02050CBEC00F0000E8D
:10062000CBEC00F03BAC2ED0D6CF4EF0D7CF4FF076
:10063000E86A4BBA010F4FB4010824E04B8A4FA47B
:100640004B9A3050365C106E31503758116E7F0E19
:100650001014206E3050365C106E31503758116EC9
:1006600010C021F011C0F3FF070EF3322132E82E43
:10067000FCD7E60ECBEC00F02050CBEC00F0215084
:10068000CBEC00F02652D8B491D026A01BD065C088
:1006900024F066C025F06FC022F070C023F0D6CFE2
:1006A00014F0D7CF15F02250145C23501558245065
:1006B00016582550175817502518D8B0800AD8B8A2
:1006C000E3EC06F026A21BD067C024F068C025F03A
:1006D00071C022F072C023F0D6CF14F0D7CF15F03E
:1006E0002250145C23501558245016582550175882
:1006F00017502518D8B0800AD8B856EC07F026A4B1
:100700001BD069C024F06AC025F073C022F074C009
:1007100023F0D6CF14F0D7CF15F02250145C23501D
:100720001558245016582550175817502518D8B06A
:10073000800AD8B8C4EC07F026A61BD06BC024F002
:100740006CC025F075C022F076C023F0D6CF14F02F
:10075000D7CF15F02250145C23501558245016584A
:100760002550175817502518D8B0800AD8B8E7EC8C
:1007700007F026A81BD06DC024F06EC025F077C00E
:1007800022F078C023F0D6CF14F0D7CF15F0225046
:10079000145C2350155824501658255017581750DC
:1007A0002518D8B0800AD8B80AEC08F00AEF01F092
:1007B0000A0E1E5CD8A47ED01F5203E11E6807D229
:1007C00051D0400E1F5C21E21F504008366E000ED3
:1007D000D8A0FF0F376E37500C0DF3CF11F0365005
:1007E0000C0DF3CF10F0F45011261050345C366E1F
:1007F00011503558376E3050365C3150375804E25E
:1008000030C036F031C037F02DD0400E1F5C05E10E
:1008100034C036F035C037F025D07F0E1F5C03E1C1
:100820001E68E1D11FD0C00E1F24366E376AFF0E3E
:10083000372237500C0DF3CF11F036500C0DF3CF9B
:1008400010F0F450112610503424366E115035201B
:10085000376E3650325C3750335804E232C036F0CF
:1008600033C037F01E682E50365C2F50375808E2E0
:10087000269236502E5C536E37502F58546EE5D06A
:1008800036502E5C37502F5808E226902E50365C9A
:10089000536E2F503758546E3AD12F50375C09E1C0
:1008A0002E50365C06E1536A546A8B8A2690269253
:1008B00012006CD01F0E1E5C0CE1116AD8901F3024
:1008C000106E5F083C6E000E11543D6E1E681200E3
:1008D0005DD0200E1E5C05E11FC050F01E681200A6
:1008E00055D0420E1E5C07E11F52D8B451D81FC02C
:1008F00028F04CD04BD0430E1E5C07E11E68400E22
:100900001F5CD8B464D942D041D0440E1E5C07E1CC
:100910001E68400E1F5CD8B466D938D037D0460E5A
:100920001E5C03E0470E1E5C06E1400E1F5CD8B45F
:1009300066D92CD02BD05A0E1E5C08E11FC03AF0AD
:10094000040E3A5CD8B03A6A21D020D0640E1E5C06
:1009500003E11FC03BF01AD0650E1E5C13E11F526D
:1009600006E0090E1F5C03E21F501008516E080ECE
:10097000515C02E20C0E516E100E515C02E30C0E43
:10098000516E04D07B0E1E5CD8B402D81E681200D3
:100990008B908B962EC036F02FC037F08B8A8A92C0
:1009A0008A903A6A3B6A266A526A12003A6A3B6A3D
:1009B000400E506E0C0E516E306A316A32683368E8
:1009C000346A800E356E2E6A2F6E700E3C6E3D6A54
:1009D0008B8A8A92899689948A90266A4A6A000E3E
:1009E00030EC00F0426E11C043F0000E30EC00F02D
:1009F000466E11C047F0D8904330116E4230106EF1
:100A0000D8901132103210504626115047228B9642
:100A1000010E30EC00F0446E11C045F0010E30ECD8
:100A200000F0486E11C049F0D8904530116E443046
:100A3000106ED890113210321050482611504922B1
:100A40008B902D902D92526A12002DA00CD02D92D9
:100A500030C02EF031C02FF030C036F031C037F04A
:100A60008B8A269012002D92000E30EC00F0426E20
:100A700011C043F04650425C4750435839E28B9ACC
:100A80008B88898650C02CF00A0E096E0A6A9390F2
:100A90008190810E026E010E036E16EC00F02E06A0
:100AA000000E2F5A2680D6CF14F0D7CF15F03C5029
:100AB0001424106E3D501520116E000E1620126E7B
:100AC000000E1720136E2C501024226E000E1120E1
:100AD000236E000E1220246E000E1320256E24C0FB
:100AE00065F025C066F022C06FF023C070F00ED014
:100AF0002D802D9230C02EF031C02FF030C036F056
:100B000031C037F08B8A26909296899612002DA2DA
:100B10000CD02D9032C02EF033C02FF02EC036F006
:100B20002FC037F026928B8A12002D90010E30ECE8
:100B300000F0446E11C045F04850445C495045589F
:100B400038E28B9A8B98898450C02CF00A0E096E7B
:100B50000A6A93908190810E026E010E036E16EC6C
:100B600000F02E4A2F2A2682D6CF14F0D7CF15F0C8
:100B70003C501424106E3D501520116E000E1620AE
:100B8000126E000E1720136E2C501024226E000ED1
:100B90001120236E000E1220246E000E1320256EED
:100BA00024C067F025C068F022C071F023C072F045
:100BB0000DD02D822D9032C02EF033C02FF02EC0DC
:100BC00036F02FC037F026928B8A899412002DB010
:100BD00007D0366A376A8986269237DF4A8002D084
:100BE00026904A8012002DB207D036683768898473
:100BF00026908DDF4A8202D026924A821200000E91
:100C000030EC00F0426E11C043F04650425C475059
:100C1000435802E22D9002D02D802D922DB01DD090
:100C20008B888B9A0A0E096E0A6A93908190810EC6
:100C3000026E010E036E16EC00F0020E45EC00F0A1
:100C4000000E30EC00F0426E11C043F04650425CA2
:100C500047504358E7E32D802D928B8A8A82640E99
:100C600045EC00F08A92010E30EC00F0446E11C0A9
:100C700045F04850445C4950455804E22D92386A8A
:100C8000396A02D02D822D902DB21FD08B988B9A6D
:100C90000A0E096E0A6A93908190810E026E010E0F
:100CA000036E16EC00F0020E45EC00F0384A392ACB
:100CB000010E30EC00F0446E11C045F04850445C29
:100CC00049504558E5E32D822D908B8A8A82640E27
:100CD00045EC00F08A92D89039323832000E382430
:100CE0002E6E800E39202F6E2EC032F02FC033F0C2
:100CF00038500008306E800E3954316E346A800EE0
:100D0000356E7F0E38144C6E38C04DF039C0F3FF8D
:100D1000070EF3324D32E82EFCD7E70ECBEC00F095
:100D20004C50CBEC00F04D50CBEC00F0000E30EC12
:100D300000F0426E11C043F04650425C47504358A9
:100D400002E22D9002D02D802D922DB03AD08B88CA
:100D50008B9A0A0E096E0A6A93908190810E026E38
:100D6000010E036E16EC00F02E06000E2F5A010E37
:100D700045EC00F0000E30EC00F0426E11C043F084
:100D8000010E45EC00F0010E30EC00F0446E11C095
:100D900045F035502F5CDDE134502E5CDAE14450F3
:100DA000485C45504958D8A08A824250465C43501E
:100DB0004758D8A08A822EC036F02FC037F08986D7
:100DC00089848B8A1200000E30EC00F0426E11C054
:100DD00043F04650425C475043580EE32D802D921D
:100DE000269089968B8A30C02EF031C02FF030C00B
:100DF00036F031C037F0120037502F5C07E1365023
:100E00002E5C04E1269089968B8A12000A0E096EE8
:100E10000A6A93908190810E026E010E036E16ECA9
:100E200000F02E5202E12F5203E02E06000E2F5A40
:100E30002C52D8A42C0636502E5C536E37502F58A7
:100E4000546E545207E15050535C04E25350505CCE
:100E5000556E01D0556A2CC009F0555062EC00F077
:100E6000566ED6CF14F0D7CF15F03C501424106E28
:100E70003D501520116E000E1620126E000E172028
:100E8000136E56501024226E000E1120236E000E99
:100E90001220246E000E1320256E24C065F025C09C
:100EA00066F022C06FF023C070F01200010E30EC2B
:100EB00000F0446E11C045F04850445C495045581C
:100EC0000EE32D822D90269289948B8A32C02EF0CB
:100ED00033C02FF032C036F033C037F01200375035
:100EE0002F5C07E136502E5C04E1269289948B8AB0
:100EF00012000A0E096E0A6A93908190810E026EAA
:100F0000010E036E16EC00F02E4A2F2A2C52D8A4A4
:100F10002C062E50365C536E2F503758546E545258
:100F200007E15050535C04E25350505C556E01D0C1
:100F3000556A2CC009F0555062EC00F0566ED6CFC1
:100F400014F0D7CF15F03C501424106E3D501520EE
:100F5000116E000E1620126E000E1720136E5650E2
:100F60001024226E000E1120236E000E1220246E1B
:100F7000000E1320256E24C067F025C068F022C043
:100F800071F023C072F0120052B003D026948A92FE
:100F90001DD0D6CF14F0D7CF15F05FC006F060C0DB
:100FA00007F006501424226E07501520236E000E01
:100FB0001620246E000E1720256E24C069F025C06F
:100FC0006AF022C073F023C074F08172120052B232
:100FD00003D026968B961DD0D6CF14F0D7CF15F020
:100FE00061C006F062C007F006501424226E07505C
:100FF0001520236E000E1620246E000E1720256E7D
:1010000024C06BF025C06CF022C075F023C076F0D0
:101010008276120052B403D026988B901DD0D6CF82
:1010200014F0D7CF15F063C006F064C007F0065087
:101030001424226E07501520236E000E1620246EF5
:10104000000E1720256E24C06DF025C06EF022C062
:1010500077F023C078F08270120080A805D0FF0ED0
:101060003E5CD8A03E2A03D03E52D8A43E0680AAB9
:1010700005D0FF0E3F5CD8A03F2A03D03F52D8A432
:101080003F063BA034D0D6CF4EF0D7CF4FF04EC066
:1010900009F04FC00AF05150E82A0A320932E82E0E
:1010A000FCD7010ED8A0E86A066E4BBC01081FE011
:1010B0004EC009F04FC00AF05150E82A0A320932F6
:1010C000E82EFCD7010ED8A0E86A4B8CE8A04B9C18
:1010D0007F0E3E14206E3E44010B216EE00ECBECE1
:1010E00000F02050CBEC00F02150CBEC00F03BA204
:1010F00034D0D6CF4EF0D7CF4FF04EC009F04FC00E
:101100000AF05150E82A0A320932E82EFCD7010EC3
:10111000D8A0E86A066E4BBE01081FE04EC009F079
:101120004FC00AF05150E82A0A320932E82EFCD7A3
:10113000010ED8A0E86A4B8EE8A04B9E7F0E3F14AC
:10114000206E3F44010B216EE10ECBEC00F02050ED
:10115000CBEC00F02150CBEC00F01200D8903E32E6
:101160003E8E80A83E9ED8903F323F8E80AA3F9E02
:101170003BA034D0D6CF4EF0D7CF4FF04EC009F0C1
:101180004FC00AF05150E82A0A320932E82EFCD743
:10119000010ED8A0E86A066E4BBC01081FE04EC0E5
:1011A00009F04FC00AF05150E82A0A320932E82EFD
:1011B000FCD7010ED8A0E86A4B8CE8A04B9C7F0EB0
:1011C0003E14206E3E44010B216EE00ECBEC00F08D
:1011D0002050CBEC00F02150CBEC00F03BA234D0FF
:1011E000D6CF4EF0D7CF4FF04EC009F04FC00AF027
:1011F0005150E82A0A320932E82EFCD7010ED8A055
:10120000E86A066E4BBE01081FE04EC009F04FC0F1
:101210000AF05150E82A0A320932E82EFCD7010EB2
:10122000D8A0E86A4B8EE8A04B9E7F0E3F14206E3C
:101230003F44010B216EE10ECBEC00F02050CBECD3
:1012400000F02150CBEC00F01200D8903E363E80EA
:1012500080A83E90D8903F363F8080AA3F903BA028
:1012600034D0D6CF4EF0D7CF4FF04EC009F04FC09C
:101270000AF05150E82A0A320932E82EFCD7010E52
:10128000D8A0E86A066E4BBC01081FE04EC009F00A
:101290004FC00AF05150E82A0A320932E82EFCD732
:1012A000010ED8A0E86A4B8CE8A04B9C7F0E3E1440
:1012B000206E3E44010B216EE00ECBEC00F020507E
:1012C000CBEC00F02150CBEC00F03BA234D0D6CFD9
:1012D0004EF0D7CF4FF04EC009F04FC00AF051503A
:1012E000E82A0A320932E82EFCD7010ED8A0E86AB3
:1012F000066E4BBE01081FE04EC009F04FC00AF059
:101300005150E82A0A320932E82EFCD7010ED8A043
:10131000E86A4B8EE8A04B9E7F0E3F14206E3F4440
:10132000010B216EE10ECBEC00F02050CBEC00F075
:101330002150CBEC00F01200E86A26B0010F26B273
:101340000109066E076A07500610D8A443D03F5023
:10135000FF08366E000ED8A0FF0F376E3634106EC1
:101360003734116E1036113610361136F80E10164D
:1013700010503424366E11503520376E3E50FF0821
:10138000406E000ED8A0FF0F416E030ED89040367D
:101390004136E82EFBD74050365E4150375A2E502A
:1013A000365C2F50375804E28B808B9625EC05F085
:1013B00036502E5C37502F5804E28B868B9087EC8A
:1013C00005F02F50375C06E12E50365C03E18B9020
:1013D0008B968B8A1200E86A26B0010F26B20109AB
:1013E000066E076A07500610D8A447D03F50FF0882
:1013F000366E000ED8A0FF0F376E3634106E3734BD
:10140000116E1036113610361136F80E10161050B7
:101410003424366E11503520376E3E50FF08406E32
:10142000000ED8A0FF0F416E4034106E4134116E93
:101430001036113610361136F80E10161050365E72
:101440001150375A2E50365C2F50375804E28B8695
:1014500025EC05F012D036502E5C37502F5804E2A0
:101460008B8087EC05F009D02F50375C06E12E50B9
:10147000365C03E18B8A8B808B863E28D8B48B96B2
:101480003F28D8B48B901200E86A26B0010F26B22C
:101490000109066E076A07500610D8A44BD03F50CA
:1014A0003E5C17E23E503F5C366E376AD8A0370686
:1014B0003634106E3734116E103611361036113640
:1014C000F80E10161050345C366E11503558376EC9
:1014D00016D03F503E5C366E376AD8A03706363499
:1014E000106E3734116E1036113610361136F80E74
:1014F000101610503424366E11503520376E2E5091
:10150000365C2F50375804E28B8625EC05F012D05C
:1015100036502E5C37502F5804E28B8087EC05F054
:1015200009D02F50375C06E12E50365C03E18B8AE0
:101530008B808B863E28D8B48B963F28D8B48B906E
:041540001200FFD7BF
:020000040030CA
:0300010006170ED1
:020005008581F3
:060008000FC00FE00F40E5
:00000001FF
